:100000000C94340018950000189500001895000015
:10001000189500001895000018950000189500002C
:10002000189500001895000018950000189500001C
:10003000189500001895000018950000189500000C
:1000400018950000189500001895000018950000FC
:1000500018950000189500001895000018950000EC
:1000600018950000189500008FEF8DBFC8EDE0ECEB
:100070004E2E84E08EBFD4E0F4E05F2EA89584B7C6
:10008000082E877F84BF88E1992780936000909332
:100090006000EEEFF3E0A0E0B1E088278D933197A8
:1000A000E9F7662438983B98339A309A89E591E0CD
:1000B000A0E0B1E08D939C93709102017068709301
:1000C00002018FEF8AB9269A279A2F9A2E9870915B
:1000D00002017F7B70930201229A209A21980E944C
:1000E00096062A9A8AE090E00E94AC062A98289800
:1000F0005A924A9287E0D2018C9381E00E94BB061B
:100100005A924A9281E0D2018C9381E00E94BB0610
:100110000E944003249682E00E9454062A980E947E
:100120004F0382E090E00E94AC062A9A19990C9441
:10013000F9002A985A924A9281E6D2018C9381E082
:100140000E94BB065A924A9285E0D2018C9381E0CC
:100150000E94BB060E944003249682E00E9454063F
:100160005A924A9287E1D2018C9381E00E94BB06A9
:100170005A924A9281E0D2018C9381E00E94BB06A0
:100180000E944003249682E00E945406AEE2B1E051
:100190000C9100FB16F00C949A0087E280930D01FD
:1001A00080E480930E015A924A9282E0D2018C93AD
:1001B00081E00E94BB060E943603229681E00E94E5
:1001C00054062A9A82E090E00E94AC0680913201A7
:1001D00080930A018091310180930B0180E090E0CF
:1001E000A0E0B1E08D939C93709102017F777093B2
:1001F0000201ABE0B1E00C9105FB16F00C94070195
:10020000709102017064709302010C940C01709162
:1002100002017F7B70930201A2E0B1E08C9186FB2A
:1002200016F40C94680180E080930C01AAE0B1E020
:100230000C9104FB16F00C94200181E080930C01DA
:10024000AAE0B1E00C9105FB16F00C942C01ACE097
:10025000B1E08C918E5F8C93AAE0B1E00C9106FB2B
:1002600016F00C943801ACE0B1E08C918C5F8C936B
:10027000AAE0B1E00C9107FB16F00C944401ACE04D
:10028000B1E08C91885F8C93ABE0B1E00C9100FB06
:1002900016F00C945001ACE0B1E08C91805F8C932F
:1002A000ABE0B1E00C9101FB16F00C945C01ACE00A
:1002B000B1E08C91805E8C93ABE0B1E00C9102FBDD
:1002C00016F00C946801ACE0B1E08C91805C8C93EA
:1002D000A2E0B1E08C9186FB16F00C94C40180E0A2
:1002E00080930C01AAE0B1E00C9104FB16F40C948D
:1002F0007C0181E080930C01AAE0B1E00C9105FB48
:1003000016F40C948801ACE0B1E08C918E5F8C9374
:10031000AAE0B1E00C9106FB16F40C949401ACE059
:10032000B1E08C918C5F8C93AAE0B1E00C9107FB5B
:1003300016F40C94A001ACE0B1E08C91885F8C9332
:10034000ABE0B1E00C9100FB16F40C94AC01ACE016
:10035000B1E08C91805F8C93ABE0B1E00C9101FB3C
:1003600016F40C94B801ACE0B1E08C91805E8C93F3
:10037000ABE0B1E00C9102FB16F40C94C401ACE0CC
:10038000B1E08C91805C8C9380910C01809308018A
:1003900080E08093090100910801093018F011F004
:1003A0000C94D4010C94E001A8E0B1E08C918A5047
:1003B0008C93A9E0B1E08C918F5F8C930C94CB016E
:1003C0000E94D40610ED0E94EC0611E00E94EC069B
:1003D0000E94D40611ED0E94EC060E940B07A3E0D8
:1003E000B1E01C930E940907A5E0B1E01C930E94B4
:1003F000E306A3E0B1E09C910E947706A3E0B1E0A0
:100400008C93A5E0B1E09C910E947706A5E0B1E055
:100410008C9380E08093040100910301093018F06F
:1004200011F00C9415020C942102A3E0B1E08C9120
:100430008A508C93A4E0B1E08C918F5F8C930C94E4
:100440000C0280E08093060100910501093018F04C
:1004500011F00C942D020C943902A5E0B1E08C91BE
:100460008A508C93A6E0B1E08C918F5F8C930C94B2
:1004700024020E94E803E1E0F0E00E945F06339965
:100480000C94AD020E94D40610ED0E94EC0611E01F
:100490000E94EC060E94D40611ED0E94EC060E9418
:1004A0000B07A3E0B1E01C930E940907A5E0B1E0AF
:1004B0001C930E94E306A3E0B1E09C910E947706A2
:1004C000A3E0B1E08C93A5E0B1E09C910E94770697
:1004D000A5E0B1E08C93A5E0B1E08C918F5F8C93A7
:1004E00000910501083111F00C94790280E08093AD
:1004F000050180E080930701A7E0B1E08C910E94A4
:100500007006A7E0B1E08C93A3E0B1E08C910E946B
:100510007006A3E0B1E08C93A5E0B1E08C910E945D
:100520007006A5E0B1E08C930E94D40610ED0E9405
:10053000EC0610E00E94EC06A7E0B1E01C910E94DE
:10054000EC06A3E0B1E01C910E94EC06A5E0B1E04E
:100550001C910E94EC060E94E30630990C941E0345
:100560000E94D40610ED0E94EC0611E00E94EC06F9
:100570000E94D40611ED0E94EC060E940B07A3E036
:10058000B1E01C930E940907A5E0B1E01C930E9412
:10059000E306A3E0B1E09C910E947706A3E0B1E0FE
:1005A0008C93A5E0B1E09C910E947706A5E0B1E0B4
:1005B0008C93A3E0B1E08C918F5F8C930091030149
:1005C0000B3318F011F00C94E7020C94EA0280E06F
:1005D0008093030180E080930701A7E0B1E08C9154
:1005E0000E947006A7E0B1E08C93A3E0B1E08C918B
:1005F0000E947006A3E0B1E08C93A5E0B1E08C917D
:100600000E947006A5E0B1E08C930E94D40610ED24
:100610000E94EC0610E00E94EC06A7E0B1E01C91FD
:100620000E94EC06A3E0B1E01C910E94EC06A5E05C
:10063000B1E01C910E94EC060E94E306A0E0B1E04C
:100640000E945806A0E0B1E00D911C910E3551E0DA
:1006500015071CF011F00C942F030C9434037091C7
:1006600002017068709302010C9496002898A8818A
:10067000B9819C91ADE0B1E00E948C06289A089562
:10068000289891E0AA81BB810E948C06A881B9813B
:100690009C91AEE2B1E00E948106289A08958AE218
:1006A00080930D0184E380930E0183E480930F0116
:1006B00080E18093100180E18093110181E08093BB
:1006C00012015A924A9286E0D2018C9381E00E94F4
:1006D000BB060E943603229681E00E94540681E206
:1006E00080930D0181E080930E015A924A9282E03C
:1006F000D2018C9381E00E94BB060E9436032296B1
:1007000081E00E94540682E280930D0181E0809393
:100710000E015A924A9282E0D2018C9381E00E94AB
:10072000BB060E943603229681E00E94540685E2B1
:1007300080930D0188E280930E015A924A9282E0E2
:10074000D2018C9381E00E94BB060E943603229660
:1007500081E00E94540681E380930D0185E080933F
:100760000E015A924A9282E0D2018C9381E00E945B
:10077000BB060E943603229681E00E94540686E260
:1007800080930D018FE080930E015A924A9282E08D
:10079000D2018C9381E00E94BB060E943603229610
:1007A00081E00E94540680E280930D018FE08093E7
:1007B0000E015A924A9282E0D2018C9381E00E940B
:1007C000BB060E943603229681E00E9454060895DB
:1007D00078E37BB92E9A2F982F9A2E9800910601D4
:1007E000003011F00C94F8037BE77BB90C943E04C5
:1007F000013011F00C94000470E37BB90C943E04BA
:10080000023011F00C9408047DE67BB90C943E0490
:10081000033011F00C94100475E77BB90C943E047E
:10082000043011F00C94180476E37BB90C943E0468
:10083000053011F00C94200477E57BB90C943E044C
:10084000063011F00C9428047FE57BB90C943E042B
:10085000073011F00C94300470E77BB90C943E041F
:10086000083011F00C9438047FE77BB90C943E04F7
:10087000093011F00C943E0477E77BB90091060132
:10088000003011F00C94460470E07BB92F982F9A39
:1008900079E37BB92E9A2F982F9A2E980091050113
:1008A000003011F00C9458047BE77BB90C949E0443
:1008B000013011F00C94600470E37BB90C949E0439
:1008C000023011F00C9468047DE67BB90C949E0410
:1008D000033011F00C94700475E77BB90C949E04FE
:1008E000043011F00C94780476E37BB90C949E04E8
:1008F000053011F00C94800477E57BB90C949E04CC
:10090000063011F00C9488047FE57BB90C949E04AA
:10091000073011F00C94900470E77BB90C949E049E
:10092000083011F00C9498047FE77BB90C949E0476
:10093000093011F00C949E0477E77BB92F982F9A19
:100940007AE37BB92E9A2F982F9A2E980091040162
:10095000003011F00C94B0047BE77BB90C94F604E2
:10096000013011F00C94B80470E37BB90C94F604D8
:10097000023011F00C94C0047DE67BB90C94F604AF
:10098000033011F00C94C80475E77BB90C94F6049D
:10099000043011F00C94D00476E37BB90C94F60487
:1009A000053011F00C94D80477E57BB90C94F6046B
:1009B000063011F00C94E0047FE57BB90C94F6044A
:1009C000073011F00C94E80470E77BB90C94F6043E
:1009D000083011F00C94F0047FE77BB90C94F60416
:1009E000093011F00C94F60477E77BB92F982F9A11
:1009F0007BE37BB92E9A2F982F9A2E9800910301B2
:100A0000003011F00C9408057BE77BB90C944E057F
:100A1000013011F00C94100570E37BB90C944E0575
:100A2000023011F00C9418057DE67BB90C944E054C
:100A3000033011F00C94200575E77BB90C944E053A
:100A4000043011F00C94280576E37BB90C944E0524
:100A5000053011F00C94300577E57BB90C944E0508
:100A6000063011F00C9438057FE57BB90C944E05E7
:100A7000073011F00C94400570E77BB90C944E05DB
:100A8000083011F00C9448057FE77BB90C944E05B3
:100A9000093011F00C944E0577E77BB92F982F9A07
:100AA0007CE37BB92E9A2F982F9A2E98A2E0B1E082
:100AB0008C9187FB16F40C947105A2E0B1E08C9147
:100AC00086FB16F00C94660574E07BB9A2E0B1E0F9
:100AD0008C9186FB16F40C946F0570E07BB90C9436
:100AE000730574E07BB92F982F9A7DE37BB92E9A1A
:100AF0002F982F9A2E98A2E0B1E08C9187FB16F4E4
:100B00000C94D40500910901003011F00C948C056F
:100B100070E07BB90C94D205013011F00C9494056F
:100B200070E37BB90C94D205023011F00C949C0553
:100B30007DE67BB90C94D205033011F00C94A4052A
:100B400075E77BB90C94D205043011F00C94AC0518
:100B500076E37BB90C94D205053011F00C94B40502
:100B600077E57BB90C94D205063011F00C94BC05E6
:100B70007FE57BB90C94D205073011F00C94C405C5
:100B800070E77BB90C94D205083011F00C94CC05B9
:100B90007FE77BB90C94D205093011F00C94D20593
:100BA00077E77BB90C94D60574E07BB92F982F9A20
:100BB0007EE37BB92E9A2F982F9A2E98A2E0B1E06F
:100BC0008C9187FB16F40C943706009108010030D5
:100BD00011F00C94EF057BE77BB90C9435060130DE
:100BE00011F00C94F70570E37BB90C9435060230D4
:100BF00011F00C94FF057DE67BB90C9435060330AB
:100C000011F00C94070675E77BB90C943506043097
:100C100011F00C940F0676E37BB90C943506053081
:100C200011F00C94170677E57BB90C943506063065
:100C300011F00C941F067FE57BB90C943506073044
:100C400011F00C94270670E77BB90C943506083038
:100C500011F00C942F067FE77BB90C943506093010
:100C600011F00C94350677E77BB90C94390674E0E3
:100C70007BB92F982F9A7FE37BB92E9A2F982F9AC2
:100C80002E98A2E0B1E08C9187FB16F40C944C06F0
:100C900076E67BB90C944E0674E07BB92F982F9AB8
:100CA0000895481A590A0895481A8827580A089535
:100CB000ED91FC91EF5FFF4FFC93EE93089588EE6A
:100CC00093E04AD03197D9F70895982F82958F7085
:100CD000805D8D939F70905D9D9388278C93089580
:100CE0004AE0082F0E94BF060295802B0895892FA5
:100CF0008F70905110F0865FFCCF08953197F1F717
:100D000008950E949D068C910E949F068D939A954E
:100D1000D1F70E949E0608950E949D068D910E9423
:100D20009F069A95D9F70E949E060895259A2498C1
:100D30002C9A239A80E58CBD0895089508958EBD60
:100D400000904D0007FEFCCF8EB50895689462F8C0
:100D50000895E89462F80895EF93FF93EE27E82B47
:100D6000E92B31F0E0EDF7E03197F1F70197D1F79A
:100D7000FF91EF910895480E8827581E0895FF931C
:100D8000881BF9E0001FFA9511F4FF910895881F60
:100D9000841B18F4840F8894F5CF0894F3CF4498FB
:100DA00045983C983D9808953D9A3C9803D03D98CD
:100DB00001D03C9AEF93FF93E6E0F0E00E947E06BC
:100DC000FF91EF9108953D9A3C9AF4DF3D98359B51
:100DD000FECFF0DF3C98EECF0894111F01C0110F39
:100DE00069F03D9A18F400003C9802C03C9A00C09B
:100DF000E1DF3D98359BFECFDDDFF1CF3D9A3C989A
:100E0000D9DF3D98359BFECFE8943499689462F819
:100E1000D1CF089401C08894331F11E03D9A3C98CB
:100E2000C9DF3D98359BFECFC5DF8894349908947F
:100E3000111FA0F73D9A379510F43C9801C03C9AD9
:0C0E4000B9DF3D98359BFECFB5DF08956B
:00000001FF
